:0200000480007A
:100000006F00C004732F2034930F8000630AFF0336
:10001000930F90006306FF03930FB0006302FF038A
:10002000170F0080130F0FFE63040F0067000F000F
:10003000732F203463540F006F00400093E19153FD
:10004000171F000023203FFC6FF09FFF732540F136
:1000500063100500970200009382020173905230F2
:10006000735000189702000093820202739052307E
:10007000B70200809382F2FF7390023B9302F0017B
:100080007390023A9702000093828201739052307B
:100090007350203073503030735040309301000063
:1000A00097020000938242F67390523013051000BD
:1000B0001315F501634C05000F00F00F93011000BC
:1000C0009308D0051305000073000000970200801C
:1000D000938242F3638E020073905210B7B2000015
:1000E000938292107390223073232030E39862F44D
:1000F00073500030970200009382420173901234D3
:10010000732540F17300203093012000930200001A
:100110001703000013030301E70203006F00000C44
:10012000170300001303C3FF639A620A93014000A0
:10013000130200001703000013030301E706030086
:10014000631E30081302120093022000E31452FED3
:100150009301500013020000170300001303430132
:1001600013000000E7060300631A300613021200B2
:1001700093022000E31252FE93016000130200007C
:100180001703000013038301130000001300000095
:10019000E7060300631430041302120093022000E8
:1001A000E31052FE93021000170300001303C30173
:1001B0006700C3FF938212009382120093821200A1
:1001C000938212009382120093821200930E4000D9
:1001D000930170006394D201631030020F00F00F9E
:1001E000638001009391110093E111009308D00501
:1001F00013850100730000000F00F00F9301100041
:100200009308D0051305000073000000731000C0B0
:1002100000000000000000000000000000000000DE
:1002200000000000000000000000000000000000CE
:1002300000000000000000000000000000000000BE
:0402400000000000BA
:1010000000000000000000000000000000000000E0
:1010100000000000000000000000000000000000D0
:1010200000000000000000000000000000000000C0
:1010300000000000000000000000000000000000B0
:081040000000000000000000A8
:040000058000000077
:00000001FF
